:020000040000FA
:1000000014280A30FB00FB0B06280B282430FC00C8
:10001000FC0B082803280800FD00FD0AFD0B112831
:10002000132801200E2808000313831606309F00B2
:1000300085018601870103138312850186018701EB
:10004000EE213322E720DC219721F2206A202920AB
:1000500020281430A1000617861686158617061666
:100060008122061386128611861306127B228714BC
:10007000071487150715851581228710071087112A
:10008000071185117B22861406148717061586151D
:100090008122861006108713061186117B22851493
:1000A0000514061605158515812285100510061202
:1000B000051185117B2287160716871507178717E5
:1000C0008122871207128711071387137B22A10B46
:1000D0002B2808000A30A100972081229B207E2235
:1000E0009F208122A3207E22A7208122AB207E2276
:1000F000AF208122B3207E22B7208122BB207E2226
:10010000BF208122C3207E22C7208122CB207E22D5
:10011000CF208122D3207E22D7208122DB207E2285
:10012000DF208122E3207E22A10B6C280800061725
:100130008616861508000613861286110800861595
:10014000061586140800861106118610080086140C
:1001500006148717080086100610871308008717F3
:1001600007178716080087130713871208008716DA
:1001700007168715080087120712871108008715D0
:1001800007158714080087110711871008008714C6
:1001900007148515080087100710851108008515BC
:1001A00005158514080085110511851008008514B2
:1001B000051406160800851005100612080006161C
:1001C0008617061708000612861306130800053066
:1001D000A1001E30A000F6211E30A0003B22A10B82
:1001E000E92808001430A10006170A30A000782280
:1001F00006130A30A000782287170A30A000782260
:1002000087130A30A000782207140A30A000782251
:1002100007100A30A000782206150A30A0007822C4
:1002200006110A30A000782206140A30A0007822B5
:1002300006100A30A000782205150A30A0007822A6
:1002400005110A30A000782286140A30A000782216
:1002500086100A30A000782285150A30A000782286
:1002600085110A30A000782287150A30A000782274
:1002700087111E30A000782286160A30A00078224E
:1002800086120A30A000782285140A30A000782255
:1002900085100A30A000782207170A30A0007822C3
:1002A00007130A30A000782205140A30A000782233
:1002B00005100A30A000782207160A30A000782224
:1002C00007120A30A000782286170A30A000782290
:1002D00086130A30A000782287160A30A000782200
:1002E00087120A30A000782206160A30A000782271
:1002F00006120A30A000782207150A30A0007822E2
:1003000007110A30A000782286150A30A000782252
:1003100086110A30A000782287140A30A0007822C3
:1003200087100A30A0007822A10BF42808000A30B8
:10033000A100061786148716871485141430A000B0
:100340007822061386108712871085103C30A00093
:100350007822861587178715851506161430A00094
:100360007822861187138711851106123C30A00070
:100370007822861606140716071405141430A000F8
:100380007822861206100712071005103C30A000D4
:100390007822061507170715051586171430A000D3
:1003A0007822061107130711051186133C30A000AF
:1003B0007822A10B992908001430A100FF30850094
:1003C000860087001430A00078228501860187010D
:1003D0009630A0007822A10BDE2908000530A1008C
:1003E0001E30A000F621A10BF02908000617782284
:1003F000061386177822861306167822061205142D
:1004000078220510851478228510051578220511AB
:100410008515782285110714782207108714782211
:10042000871007157822071187157822871107167C
:100430007822071287167822871207177822071367
:1004400087177822871306147822061086147822DC
:1004500086100615782206118615782286118616D2
:100460007822861208000530A1001E30A0003B2231
:10047000A10B352A08000617782206138616782263
:1004800086128615782286110615782206118614A2
:100490007822861006147822061087177822871390
:1004A00007177822071387167822871207167822F3
:1004B00007128715782287110715782207118714EC
:1004C0007822871007147822071085157822851165
:1004D00005157822051185147822851005147822D7
:1004E0000510061678220612861778228613080051
:1004F00020080C20080064300C20080028300C2054
:0805000008000A300C2008007D
:084000000100090004000900A1
:02400E00313F40
:00000001FF
